:1010000039C000006EC000006CC000006AC0000063
:1010100068C0000066C0000064C0000062C000003C
:1010200060C000005EC000005CC000003DC5000064
:1010300058C0000056C0000054C0000052C000005C
:1010400050C000004EC00000B9C100004AC00000FE
:1010500048C0000046C0000044C0000042C000007C
:1010600040C000003EC000003CC000003AC000008C
:1010700038C0000011241FBECFEFD2E0DEBFCDBFCD
:1010800004B603FE19C080917F01909180018234E3
:101090009C4D91F484B7877F84BF88E10FB6F894A4
:1010A00080936000109260000FBE10928001109239
:1010B0007F01E0E0F0E0099511E0A0E0B1E0EEE7AB
:1010C000FDE102C005900D92A236B107D9F721E0EB
:1010D000A2E6B1E001C01D92AF37B207E1F738D107
:1010E0004CC68ECF8823A9F09091F20091110DC0CB
:1010F0009091E8009B7F9093E8009091E80092FD2A
:1011000006C09EB39111F9CF04C09091F1008150B7
:10111000E9CF089530916F0120916E0190916D019A
:1011200080916C019093640180936501C901909353
:1011300062018093630108951F93CF93DF93CDB72E
:10114000DEB727970FB6F894DEBF0FBECDBF9091E4
:10115000740180916A019923D1F0843049F480911F
:101160006B01811108C080916C018F3F21F45AC03E
:10117000853009F4ADC08AE08093000183E080935C
:1011800072018091EB0080628093EB00D7C08430C5
:1011900009F448C028F4813051F08330F1F0CEC01A
:1011A000853009F495C0863009F4BCC0C7C01091E1
:1011B0006B01123008F0C2C0ADDF11110CC080917C
:1011C00064019091650123E0FC0120935700E895AC
:1011D00007B600FCFDCF85E007C080916B01982F1A
:1011E0009D7F29F497DF89E080930001A7C08130BB
:1011F00009F0A4C0E0E0F0E084918F3F69F0109224
:101200006601F0936501E09364018AE08093000138
:1012100085E08093720192C03196E11520E1F207DA
:1012200059F78CC080916B01833071F581E0809318
:101230007301809170019091710120916C01892B53
:1012400061F0213009F07AC090916F0180916E01B8
:10125000909367018093680171C0211112C082E4EC
:101260009CED9093800180937F012CE088E190E0D9
:101270000FB6F894A895809360000FBE209360008D
:101280005DC0109201015AC0811158C080916C015B
:101290008F3F09F053C0E0E0F0E083E095E08093F9
:1012A0005700E89507B600FCFDCF90935700E895EE
:1012B00007B600FCFDCFE058FF4FE11520E1F20733
:1012C00071F781E180935700E8951092740136C060
:1012D00080E28D838CED8E838BEF8F8388E589830D
:1012E0008EE18A8383E98B8389E88C8320916C016A
:1012F00080916B01811105C0FE01E20FF11D858116
:101300000EC08130D9F4822F90E0FE01203610F417
:10131000BF9702C0EC55F109E80FF91F8081809357
:1013200069010CC080916B01833041F480916C01A4
:10133000811104C080916D018093660127960FB6DC
:10134000F894DEBF0FBECDBFDF91CF911F910895FE
:1013500084B7877F84BF88E10FB6F89480936000DC
:10136000109260000FBE90E080E80FB6F894809372
:101370006100909361000FBEC1E0C5BF82E085BFF0
:1013800084D3C0936F0083E0809381007894809130
:101390000101882311F0D3D4FACF80917301811118
:1013A000FACF2AD310926F001092810081E085BF9E
:1013B00015BEE0916701F091680109951F920F92A7
:1013C0000FB60F9211240F900FBE0F901F9018951B
:1013D000CF92DF92EF92FF920F931F93CF93DF9301
:1013E000809177018F77813209F0E7C180917D018B
:1013F00090917E01909371018093700180917801AA
:10140000833009F49BC158F48130D1F0823009F067
:10141000D4C18091E800877F8093E80003C18530C4
:1014200009F4B2C108F4A8C1863009F0C6C18091A0
:10143000E800877F8093E80082E080930001B4C1D8
:101440008091E800877F8093E80080917301882372
:1014500019F072DE10927301809170019091710108
:10146000009741F12091E80022FD04C02EB3211124
:10147000F9CFA3C12091F10020936A0101979093C5
:10148000710180937001EBE6F1E08091F200882316
:1014900081F08091F10081938091700190917101B0
:1014A0000197909371018093700181E0E037F80714
:1014B00061F742DE80910001853009F0ABC0809178
:1014C000700190917101892B21F482E080930001D9
:1014D000A1C08AE107DEE0906401F09065018E2DE5
:1014E0008F7100DE00916201109163010F5F1F4F49
:1014F0000E191F0980916B01811182C0E801D695F8
:10150000C795C70120916601A22FB0E08C019D0113
:10151000F12CEE24E39465E0D62E73E0C72E2097DD
:1015200009F442C04091F2004423D1F02197709118
:10153000F1006091F100472F562FFC010A01E09263
:101540005700E8951124F394AC01BD014E5F5F4F45
:101550006F4F7F4FDB01CA01F0E4FF120EC00FC0D6
:101560004091E8004B7F4093E8004091E80042FD45
:10157000DDCF4EB34111F9CF20C1209781F6F8019C
:10158000D0925700E89507B600FCFDCF209709F4EC
:10159000C6CFFA01C0925700E89507B600FCFDCF10
:1015A0008A019B01F12CBBCF809162019091630174
:1015B000909365018093640181E180935700E895E1
:1015C00027C08091F200811109C08091E8008B7FD3
:1015D0008093E8008091E80082FF16C00150110955
:1015E0006091F1008091640190916501B8D3809180
:1015F0006401909165010196909365018093640167
:1016000001151105F1F604C08EB38111E3CFD5C0E9
:1016100080E168DD8091E8008B7F8DC08EB38823E8
:1016200009F4CBC08091E80080FFF8CF80910001E1
:10163000893091F08A3059F480916B01813039F40E
:1016400090916401809165019093F10002C08091B6
:1016500069018093F1006CC0409164015091650173
:1016600020916201309163012F5F3F4F241B350BA6
:1016700080916B01811131C0CA0140916601A42F94
:10168000B0E03695279521153105F1F04091F20033
:10169000403269F44091E8004E7F4093E800409169
:1016A000E80040FD04C04EB34111F9CF86C0FC01F3
:1016B000459154914093F1005093F1000296A11D81
:1016C000B11D21503109DFCF8091620190916301FA
:1016D000909365018093640128C0823031F5E9015F
:1016E000209719F18091F200803269F48091E8002E
:1016F0008E7F8093E8008091E80080FD04C08EB367
:101700008111F9CF5AC080916401909165011FD376
:101710008093F1008091640190916501019690930E
:101720006501809364012197DBCF82E08093000103
:101730008091E8008E7F8093E80036C08091E800B9
:10174000877F8093E8008091E80080FD04C08EB31D
:101750008111F9CF32C0809172018093F100109213
:10176000F1001092F1001092F1008091000180933D
:10177000F1001092F100DCCF8091E800877F809328
:10178000E8001092720110C08091E800877F80937A
:10179000E8008091E80080FD04C08EB38111F9CF8C
:1017A0000CC08091000155CFDF91CF911F910F9117
:1017B000FF90EF90DF90CF9000C1DF91CF911F910C
:1017C0000F91FF90EF90DF90CF900895292F30E098
:1017D0002230310539F02330310549F0213031050F
:1017E00061F410C08BE190E024E331E01EC0882357
:1017F00071F0813089F08230A1F080E090E020E04B
:1018000030E013C082E190E02FE431E00EC084E0CC
:1018100090E020E331E009C088E190E026E131E08A
:1018200004C082E190E022E031E0FA0131832083BC
:10183000089507B600FCFDCFF999FECF23E0FB0128
:1018400020935700E89507B600FCFDCF81E1809317
:101850005700E895089507B600FCFDCFF999FECF33
:1018600025E0FB0120935700E89507B600FCFDCF6B
:1018700081E180935700E895089507B600FCFDCFFD
:10188000F999FECF21E0FB010A0120935700E8956A
:101890001124089521E2FC012093570084910895BA
:1018A00029E0FC012093570084910895E1E0F0E0E5
:1018B00089E0809357008491089507B600FCFDCF1E
:1018C000F999FECF809599E0E1E0F0E0082E909341
:1018D0005700E895089520917D0130917E012617EB
:1018E000370748F06115710539F42091E8002E7F23
:1018F0002093E80001C0B90120E061157105C9F12C
:101900003EB3332309F442C0353009F441C030916D
:10191000E80033FD3FC03091E80032FF06C08091FF
:10192000E80082FF29C080E008953091E80030FF90
:10193000E4CF2091F20030E0FC01281B390BCF01ED
:10194000820F931F6115710549F08032910530F4C3
:1019500081918093F10061507109F1CF21E080976E
:1019600009F020E08091E8008E7F8093E800CF01AD
:10197000C4CF2111C5CFD3CF8EB3882339F08530A2
:1019800039F08091E80083FFCACF04C082E0089557
:1019900083E0089581E00895EBEEF0E080818160BE
:1019A0008083EDEEF0E010826093EC004083809144
:1019B000EE00881F8827881F08958091770187FD92
:1019C00005C08091E80080FF0DC010C08091E80044
:1019D00082FD04C08EB38111F9CF08958091E80093
:1019E0008B7F07C08EB38111ECCF08958091E80002
:1019F0008E7F8093E800089551D053D0E0EEF0E060
:101A0000808181608083E8EDF0E080818F77808342
:101A100019BCE3E6F0E0808181608083109276015A
:101A200008953CD03ED08091D8008F778093D80025
:101A30008091D80080688093D8008091D8008F7DF5
:101A40008093D80084E089BD86E089BD09B400FE9A
:101A5000FDCF1EBA1092750142E260E080E09CDF8B
:101A60008091E1008E7F8093E1008091E2008160AF
:101A70008093E2008091E20088608093E200809190
:101A8000E0008E7F8093E0000895E3E6F0E080813F
:101A90008E7F808381E080937601C3CF1092E20035
:101AA00008951092E10008951F920F920FB60F92C1
:101AB00011242F933F934F935F936F937F938F9353
:101AC0009F93AF93BF93EF93FF938091E10080FFCB
:101AD00016C08091E20080FF12C08091E2008E7FEC
:101AE0008093E2008091E20080618093E200809127
:101AF000D80080628093D80019BC1EBA1FD1809193
:101B0000E10084FF2EC08091E20084FF2AC084E0BF
:101B100089BD86E089BD09B400FEFDCF8091D80063
:101B20008F7D8093D8008091E1008F7E8093E100CB
:101B30008091E2008F7E8093E2008091E2008160DC
:101B40008093E20080917501882311F084E007C042
:101B50008091E30087FF02C083E001C081E08EBB7B
:101B6000EDD08091E10083FF21C08091E20083FFEE
:101B70001DC08091E100877F8093E10082E08EBBF1
:101B8000109275018091E1008E7F8093E100809139
:101B9000E2008E7F8093E2008091E200806180937A
:101BA000E20042E260E080E0F7DEC8D0FF91EF9112
:101BB000BF91AF919F918F917F916F915F914F9165
:101BC0003F912F910F900FBE0F901F9018951F936C
:101BD000CF93DF9300D0CDB7DEB7E7E7F1E0809198
:101BE000F100819381E0EF37F807C9F7F1DB8091CD
:101BF000E80083FF8FC09091770180917801863053
:101C0000E1F128F4882351F08530B1F083C08830A9
:101C100009F453C0893009F462C07CC09D7F9038BC
:101C200009F078C08091E800877F8093E8001092E7
:101C3000F1001092F1004CC091116CC0109179012B
:101C40001F778091E3008078812B8093E30080915F
:101C5000E800877F8093E800B0DE8091E80080FF95
:101C6000FCCF8091E30080688093E300112311F0A2
:101C700083E001C082E08EBB4DC09058923008F0E6
:101C800049C0AE014F5F5F4F60917B018091790148
:101C900090917A019BDD009709F43CC02091E80007
:101CA000277F2093E800BC0189819A8114DE80910E
:101CB000E8008B7F8093E8002DC0903859F5809123
:101CC000E800877F8093E800809175018093F100A0
:101CD0008091E8008E7F8093E8006FDE1BC0911139
:101CE00019C0909179019230A8F48091E800877F23
:101CF0008093E8009093750160DE809175018111F9
:101D000004C08091E30087FF02C084E001C081E04D
:101D10008EBB14D08091E80083FF0AC08091E80058
:101D2000877F8093E8008091EB0080628093EB00D6
:101D30000F900F90DF91CF911F91089508958EB36A
:101D4000882321F08091E80083FD41CF0895F9991F
:101D5000FECF92BD81BDF89A992780B50895262FB0
:101D6000F999FECF1FBA92BD81BD20BD0FB6F89480
:0E1D7000FA9AF99A0FBE01960895F894FFCFE3
:101D7E00020112034C0055004600410020004400B1
:101D8E0046005500000018034400650061006E0017
:101D9E002000430061006D006500720061000000CC
:101DAE000403090409021B0001010080320904002A
:101DBE000000FE0102000921030000000C100112B8
:101DCE0001100100000020EB03EE2F0000010200C5
:021DDE00010002
:101FA00048CC59CC6ACC76CC7BCC80CC86CC0895FE
:081FB0000895089508950895B5
:101FE000DFCFDFCFDFCFDFCFDFCFDFCFDFCFDFCF81
:081FF000DFCFDFCFDFCFDFCF31
:081FF8000010000010DFFBDC0B
:0400000300001000E9
:00000001FF
